:100000008316043085000030860083129C008F0028
:100010009F13D12882070334073406340434023492
:10002000063407340334053402340234033405340F
:1000300004340234073406340734043403340234FD
:1000400005340734063403340234023403340434F0
:1000500005340434033407340434063407340234DA
:100060000334043405340634013400309100083080
:1000700092001C30930008309400003095009B28BB
:100080000330910003309200003093006030940000
:10009000603095009B28033091000B3092001C309B
:1000A000930068309400603095009B286330910085
:1000B0006330920000309300633094006330950009
:1000C0009B28633091006B3092001C3093006B30A2
:1000D0009400633095009B289F1B79286B3091001A
:1000E0006B309200003093006B3094006B309500C1
:1000F0009B288F0B7D288F0A6E28851400008510A1
:100100006B30860090206B30860090200030860097
:1001100090206B30860090206B3086009020080085
:100120000A308D0060308E00803086068E0B962857
:100130008D0B9228B62885140000851011088600C2
:10014000AE2012088600AE2013088600AE201408E8
:100150008600AE2015088600AE20080004308D0011
:100160008E0BB0288D0BB0280030860005140000DF
:10017000051008001C080A209D009D0BC2280030B5
:100180009C00BA289D0BC52835289D0BC8284028FF
:100190009D0BCB284B289D0BCE2856289D0B6C28F9
:1001A00061288F1605309E0010308C00BA208C0B11
:1001B000D6289C0A9E0BD4289F17BA20051DDD283F
:0401C0009F13D12890
:00000001FF
